:100000000218DFEFD39402400122EF652860178FBA
:1000100028E52814600E14600B240270097527016E
:10002000C2028002D203D322AF3A220217B8121BB7
:10003000C5D322021E0BE4F567F566F565F564D2BB
:10004000092232021700121BC5D32202131E121AF4
:1000500043D32202170090E781E090E7C1F090E6D9
:100060008DE0FF90E780E06F6002C32290E782E0BE
:100070001215AB010100022B0102360202410301FD
:100080000414011F15014516016F1E01811F01BFD8
:100090002002493202613302783402923502ED3691
:1000A000031E3703A03803B63903C63A03DC3B030B
:1000B000EC3C04013D04113E04263F043640044B51
:1000C00041045B42047743048744049A4504B746DD
:1000D00004CA4704E74804FD49051A4A02B54B0122
:1000E000D86401DD6501E46601E96701EE6801FDA0
:1000F0006902236A05A86C06036D06AA6E00000655
:10010000D902023390E7C07407F090E7C214F0A35D
:10011000740AF0A37401F0A3F0A374040205FA902A
:10012000E7C07407F090E7C214F090E680E030E793
:10013000047F0180027F0090E7C3EFF0E4A3F0A307
:10014000F0A30205FA90E7C07407F090E7C214F03C
:10015000AD6BAF05EFA3F0E56AA3F0FEAD69AC6847
:100160007810121584AC06EFA3F0ECA30205FA9008
:10017000E7C07404F090E7C27406F0A37478020438
:100180006E90E7C07404F090E7C27406F090E783C5
:10019000E02408901F87F07E1F7F87AB07AA067DAB
:1001A000017F50121CA27E1F7F87AB07AA067D012C
:1001B0007F50121C86901F87E090E7C302046E9068
:1001C000E783E02408901F88F090E784E0901F897F
:1001D000F07E1F7F88020698121AE48056120D24C2
:1001E000D204804F120D1B804A120D1E804590E7ED
:1001F00083E0FF120D3A8E538F5402027F90E78402
:10020000E0755300F554755400F55390E783E042D0
:1002100054535301A3E0C313FFAD54AC53120D7CF0
:100220000206D4121D4B1211BFD32212002E40031E
:100230000206D90206D412004640030206D902067D
:10024000D4121D4B12004ED322121E0F8E538F5408
:1002500090E7C07404F090E7C27406F0EFA30204C4
:100260006E90E783E0755300F554FFAE531216FB12
:1002700040030206D90206D4121E138E538F5490E7
:10028000E7C07405F090E7C204F0EFA3F0E5530275
:1002900004F890E784E0755300F554FE90E783E09E
:1002A000FDEEF553EDF554FFAE53121E064003026A
:1002B00006D90206D48567588566578565568564D4
:1002C0005590E7C07407F090E7C214F0E558FFE5D9
:1002D00057FEAC06EFA3F0ECA3F0AD56AC5578108A
:1002E000121584AC06EFA3F0ECA30205FA121DC7A9
:1002F0008F588E578D568C5590E7C07407F090E755
:10030000C214F0AC06EFA3F0ECA3F0AD56AC5578F8
:1003100010121584AC06EFA3F0ECA30205FA90E7E7
:1003200086E0FFE48F58F557F556F555AE57AD56B4
:10033000AC557808121598A804A905AA06AB079031
:10034000E785E0FFEB4FF558EAF557E9F556E8F594
:1003500055AF587808121598A804A905AA06AB0746
:1003600090E784E0FFEB4FF558EAF557E9F556E8DA
:10037000F555AF587808121598A804A905AA06AB38
:100380000790E783E0FFEB4FF558EAF557E9F5569C
:10039000E8F555AF58121DBD40030206D90206D438
:1003A00090E7C07404F090E7C27406F01200289041
:1003B000E7C3EF02046E90E783E0FF121E174003CD
:1003C0000206D90206D490E7C07404F090E7C27424
:1003D00006F0121E1F90E7C3EF02046E90E783E061
:1003E000FF121C6940030206D90206D490E7C074CC
:1003F00004F090E7C27406F0121E2290E7C3EF806B
:100400006D90E783E0FF12000340030206D9020665
:10041000D490E7C07404F090E7C27406F0121E2571
:1004200090E7C3EF804890E783E0FF121D9D4003F3
:100430000206D90206D490E7C07404F090E7C274B3
:1004400006F0121E2890E7C3EF802390E783E0FFB9
:10045000121E1B40030206D90206D490E7C07404A2
:10046000F090E7C27406F0121E2B90E7C3EFF090F5
:10047000E68F7404F0D32290E783E0FF121DA840BA
:10048000030206D90206D490E7C07405F090E7C2D3
:1004900004F0E532A3F0E531805E90E784E0755327
:1004A00000F554FE90E783E0FDEEF553EDF554853D
:1004B0005331F5320206D490E7C07405F090E7C2DC
:1004C00004F0E537A3F0E536802E90E784E075531D
:1004D00000F554FE90E783E0FDEEF553EDF554850D
:1004E0005336F5370206D490E7C07405F090E7C2A2
:1004F00004F0E535A3F0E534A3F00205A090E7840D
:10050000E0755300F554FE90E783E0FDEEF553ED02
:10051000F554855334F5350206D4E52AF4704A9033
:100520001F8A04F0A37418F07E1F7F8AAB07AA0607
:100530007D027F48121CA27E1F7F8AAB07AA067D20
:10054000017F48121C86901F8AE0B41805752A01A5
:100550008003E4F52AE4901F8AF07E1F7F8AAB07B0
:10056000AA067D017F48121CA290E7C07405F09096
:10057000E7C204F0E52A601F7E1F7F8CAB07AA0646
:100580007D027F48121C86901F8CE0FCA3E090E760
:10059000C3F0ECA3F08009E490E7C3F0A3749DF0EE
:1005A00090E68F7405F0D322E4901F8EF090E7C0A0
:1005B0007407F090E7C214F0E4901F8FF07E1F7F65
:1005C0008FAB07AA067D017F50121CA27E1F7F8F72
:1005D000AB07AA067D087F50121C86901F90E09002
:1005E000E7C3F0901F91E090E7C4F0901F92E09075
:1005F000E7C5F0901F93E090E7C6F090E68F740790
:10060000F0D322E4901F97F0A374C0F07E1F7F9771
:10061000AB07AA067D027F50121CA27F50121A7AE5
:10062000901F977401F090E783E0901F98F07E1F71
:100630007F97AB07AA067D027F50121CA27F501243
:100640001A7A901F977402F090E784E0901F98F058
:100650007E1F7F97AB07AA067D027F50121CA27FE8
:1006600050121A7A901F977403F090E785E0901F5C
:1006700098F07E1F7F97AB07AA067D027F50121C61
:10068000A27F50121A7A901F977404F090E786E0C8
:10069000901F98F07E1F7F97AB07AA067D027F50C0
:1006A000121CA27F50121A7A802AE4F559901F99E1
:1006B000E559F0A374FFF07E1F7F99AB07AA067D72
:1006C000027F50121CA27F50121A7A0559E559C3B5
:1006D000940840D9121D4BD322C322200103020AE1
:1006E000BFE53B14B410004003020ABF9006FA7540
:1006F000F003A4C58325F0C5837302072A0207C946
:1007000002086302089F020ABF0208DC02095102C4
:1007100009720209AB0209CD0209EC0208210207A5
:10072000BD02093702094302091DE490E671F0F5A4
:10073000A075B4FF90E672F0F5B175B6FF00000049
:1007400090E6047480F00000007406F0000000E4FD
:10075000F0000000D200753B0290E680E030E71B1D
:1007600090E60174EAF0E5337008752E70752D1768
:100770008044E4752EB8752D0B803B90E60174AA79
:10078000F0E47FE87E03FDFCAB41AA40A93FA83E10
:10079000C312155D5019C374E89541FF7403954069
:1007A000FEE4953FFDE4953EFC121D92753B0DE481
:1007B000752E40752D1FF52CF52B020ABF2009035D
:1007C000020ABF753B02020ABF121C0AE5BB20E702
:1007D00003020ABF120D0C85636B85626A8561692D
:1007E000856068AF41AE40AD3FAC3EEC4D4E4F60D2
:1007F00003121D92E53545346021E538B4011CAF84
:100800002EAE2DAD2CAC2BAB41AA40A93FA83ED3B8
:1008100012155D4006753B0C020ABFE53D70418034
:1008200039C3E5419567FFE5409566FEE53F95656F
:10083000FDE53E9564FCAB2EAA2DA92CA82BC31276
:1008400015734003020ABF856325856224856123F1
:10085000856022120CCEE53D7006753B03020ABF8F
:10086000020A6BE47FB87E0BFDFCAB67AA66A96544
:10087000A864C31215735021120D1BE47F527E032E
:10088000FDFCAB67AA66A965A864C3121573400393
:10089000020ABF121C0A020A6B120D1E020ABF30A6
:1008A000091530000985362F85373002094B85340C
:1008B0002F85353002094BE47F64FEFDFCAB67AA4F
:1008C00066A965A864D31215735003020ABFE53800
:1008D000B40106200003020ABF020A70E5AC30E151
:1008E00039E5336005E53AB40204E4FF80027F0194
:1008F000121D82121CBEE53AB40203121CBE90E621
:1009000080E030E703120D2490E6D17401F000007E
:100910000075BB06753B07020ABF0209C7E53545EE
:10092000347005E53AB402047F0280027F03121D91
:1009300082753B0E020ABF90E6F1E0F529753B0F88
:10094000020ABFE5BB20E703020ABF753B06020AA5
:10095000BFE5BB20E703020ABF120D21E532453196
:10096000600AAE31AF32E4FCFD121D92753B080205
:100970000ABFE5AC30E003020ABF90E680E030E752
:100980001300000090E6987402F0000000E490E686
:1009900099F08011000000E490E698F000000090CB
:1009A000E6997440F0753B09020ABFE5AA20E4030A
:1009B000020ABF200903020ABFE530153070021594
:1009C0002FE530452F601F753B10020ABFE5AC30A4
:1009D000E003020ABF00000090E6987402F00000F5
:1009E00000E490E699F0753B0B020ABF90E6A5E0A3
:1009F00054706003020ABF200003020AB1E53545C6
:100A0000347003020AB1E53864017069AF2EAE2D6F
:100A1000AD2CAC2BAB41AA40A93FA83EC312155D3B
:100A20004032E5412464FFE43540FEE4353FFDE417
:100A3000353EAB07AA06A905F8C3E5639525FFE592
:100A4000629524FEE5619523FDE5609522FCD312B5
:100A50001573501CC200120CCE90E680E020E70B0C
:100A60007FE87E037D007C00121D92753B04804F61
:100A7000121CBE804AC200753B0290E680E020E76F
:100A80003EE47FE87E03FDFCAB41AA40A93FA83EBF
:100A9000C312155D5029C374E89541FF7403954056
:100AA000FEE4953FFDE4953EFC121D92753B0D80E2
:100AB0000E753B01C201E5287005752701D20220A1
:100AC0000203020B46E52724FE600C146043146009
:100AD0004E24037071D200120D0C300013121BE96A
:100AE00085362F853730E5354534600FC200800BE1
:100AF000120CCE85342F853530D200E53545347063
:100B000005E53AB402047F0280027F03121D828051
:100B100024121CBE90E6F1E0F5297527048027E534
:100B2000BB30E722120D0CE53015307002152FE5B1
:100B300030452F6005752703800C300306C202C2C2
:100B4000038003752702E5BA20E123120056401204
:100B500090E7C07403F090E7C27415F090E68F74CC
:100B600003F000000090E68D7480F0000000220089
:100B70000022120B6F0000227808D8FE22780CD8D1
:100B8000FE227810D8FE227818D8FE22C2AFC28486
:100B9000120B6FD282120B6FC286120B6FD28112B0
:100BA0000B6FC282120B6FD284120B6FC281120BB9
:100BB0006FD286120B6FD2AF22C2AFC286120B7DEC
:100BC000D281120B7DC282120B72D284120B7DC2B3
:100BD00081120B7DD286120B72C284120B7DD282DF
:100BE000120B72D2AF22C2AF7580BD120B6FC282E0
:100BF000120B6F7580FB120B6FC284120B6FD282C7
:100C0000120B6F7580ADD284120B6FD2AF22C2AFC0
:100C1000D281C284120B82120B72C283120B78D261
:100C200083120B72C281120B6FD282120B6FC286BB
:100C3000120B6FD281120B6FC282120B6FD2841211
:100C40000B6FC281120B6FD286D2AF22C2AFC286A7
:100C5000120B72D281120B7DC282120B7DD28412D2
:100C60000B87C281120B72D286120B72C284120BD6
:100C700087C28500000000D282120B82120B82D242
:100C800085120B87120B87D2AF22C2AF7580BD12BF
:100C90000B6FC282120B6F7580FB120B6FC2841236
:100CA0000B6FD282120B6F7580ADD284120B6FC2A4
:100CB00082120B87120B87758091D282120B7212EF
:100CC0000B6F7580BD120B87120B87D2AF22C2AF9C
:100CD000D281C284120B82120B72C285120B78D29F
:100CE00085120B72C281120B6FD282120B6FC286F9
:100CF000120B6FD281120B6FC282120B6FD2841251
:100D00000B6FC281120B6FD286D2AF22C2AFC280EC
:100D1000120B7D120B7DD280D2AF22D28722C287E6
:100D200022D2B522C2B522D2B5EE600678FFD8FE37
:100D3000DEFAEF6002DFFEC2B522C2B0C2B4C2B1B9
:100D4000D2B2D2B0C2B0EFC4337F033392B2D2B0CA
:100D5000C2B0DFF7C2B2D2B0C2B0D2B0C2B0D2B06D
:100D6000C2B0D2B4E4A2B333FED2B0C2B07F08A204
:100D7000B333D2B0C2B0DFF7D2B1FF22C2B0C2B437
:100D8000C2B1C2B2D2B0C2B0EFC4337F033392B2A9
:100D9000D2B0C2B0DFF7C2B2D2B0C2B0D2B0C2B02D
:100DA000D2B0C2B0EC1392B2D2B0C2B0ED7F083371
:100DB00092B2D2B0C2B0DFF7D2B12290E6B9E07001
:100DC00003020E6C147003020EE924FE7003020F7E
:100DD0006C24FB7003020E66147003020E60146034
:100DE0007314607624056003020FCB121E32400399
:100DF000020FD790E6BBE024FE602214603324FD8E
:100E0000601114602224067048E50A90E6B3F0E50C
:100E10000B8037E51290E6B3F0E513802DE50C90DA
:100E2000E6B3F0E50D8023E50E90E6B3F0E50F8024
:100E30001990E6BAE0FF121B74AA06A9077B01EA23
:100E4000494B600DEE90E6B3F0EF90E6B4F0020F80
:100E5000D7020FD0121D70020FD7121DEA020FD752
:100E6000121DE2020FD7121D5E020FD7121E344070
:100E700003020FD790E6B8E0247F601514601924B0
:100E8000027063A205E43325E0FFA207E4334F803C
:100E900041E490E740F0803F90E6BCE0547EFF7E66
:100EA00000E0D394807C0040047D0180027D00EC52
:100EB0004EFEED4F24B3F582741D3EF583E493FF9F
:100EC0003395E0FEEF24A1FFEE34E68F82F583E058
:100ED000540190E740F0E4A3F090E68AF090E68BAE
:100EE0007402F0020FD7020FD0121E364003020F19
:100EF000D790E6B8E024FE601624026003020FD704
:100F000090E6BAE0B40105C205020FD7020FD090F7
:100F1000E6BAE0705590E6BCE0547EFF7E00E0D378
:100F200094807C0040047D0180027D00EC4EFEED4B
:100F30004F24B3F582741D3EF583E493FF3395E0AF
:100F4000FEEF24A1FFEE34E68F82F583E054FEF03D
:100F500090E6BCE05480131313541FFFE0540F2F8E
:100F600090E683F0E04420F0806D8064121E3850DB
:100F70006690E6B8E024FE60192402705A90E6BA42
:100F8000E0B40104D205804F90E6BAE06402604705
:100F9000803E90E6BCE0547EFF7E00E0D394807CEF
:100FA0000040047D0180027D00EC4EFEED4F24B335
:100FB000F582741D3EF583E493FF3395E0FEEF2444
:100FC000A1FFEE34E68F82F5838008121E3A5007A7
:100FD00090E6A0E04401F090E6A0E04480F022E436
:100FE000F54EF54DF54CF54B90E600E054E7441016
:100FF000F0C208C205C207C206E4F5A075B4FF122C
:1010000014267E167F008E0A8F0B7512167513122A
:1010100075081675091C7510167511587514167516
:10102000159490E680E030E70E85080C85090D8563
:10103000100E85110F800C85100C85110D85080E82
:1010400085090FEE54E07003021159754F00755079
:10105000807E167F008E518F52C374B89FFF741626
:101060009ECF2402CF3400FEE48F4A8E49F548F526
:1010700047F546F545F544F543AF4AAE49AD48ACB2
:1010800047AB46AA45A944A843C31215735026E5A9
:10109000502546F582E54F3545F58374CDF0E5469C
:1010A0002401F546E43545F545E43544F544E43599
:1010B00043F54380C4E4F546F545F544F543AF4AAE
:1010C000AE49AD48AC47AB46AA45A944A843C312B4
:1010D00015735033E5522546F582E5513545F583C4
:1010E000E0FFE5502546F582E54F3545F583EFF005
:1010F000E5462401F546E43545F545E43544F54437
:10110000E43543F54380B7854F0A85500B740024BE
:1011100080FF741634FFFEC3E5139FF513E5129E9E
:10112000F512C3E50D9FF50DE50C9EF50CC3E50F1B
:101130009FF50FE50E9EF50EC3E5099FF509E5083D
:101140009EF508C3E5119FF511E5109EF510C3E566
:10115000159FF515E5149EF514D2E843D82090E6C6
:1011600068E04409F090E65CE0443DF0D2AF90E6E0
:1011700080E020E105D20A1215D190E680E054F714
:10118000F0538EF8C208300605120DBBC2063008B7
:1011900029121E2E5024C208121BA020051690E60C
:1011A00082E030E704E020E1EF90E682E030E60400
:1011B000E020E0E4121B48121E301206DB80C7E478
:1011C000F55EF55FF55CF55D90E6A5E020E3F9E4FA
:1011D000F55AF55BC3E55A6480948250517400253A
:1011E0005BF58274F8355AF583E55FF0E55EFF74D0
:1011F00001255BF58274F8355AF583EFF074792593
:101200005FF55FE4355EF55EFEAF5F3395E0FDFCB4
:10121000E47B3C7AFFF9F8C312155D7004F55EF5C6
:101220005F7402255BF55BE4355AF55A80A6E55DEF
:10123000B41515E55CB4021090E6987401F0000056
:101240000090E6997458800D90E6987402F00000C2
:1012500000E490E699F0000000055DE55D70020590
:101260005C64167004E55C640260030211C8E4F576
:101270005EF55FF55CF55D90E6A5E020E3F9E4F549
:101280005AF55BC3E55A6480948250517400255B23
:10129000F58274F8355AF583E55FF0E55EFF740179
:1012A000255BF58274F8355AF583EFF07479255F84
:1012B000F55FE4355EF55EFEAF5F3395E0FDFCE47F
:1012C0007B3C7AFFF9F8C312155D7004F55EF55F9B
:1012D0007402255BF55BE4355AF55A80A6E55DB4EA
:1012E0001315E55CB4021090E6987401F00000005C
:1012F00090E6997420800D90E6987402F00000004A
:10130000E490E699F0000000055DE55D7002055C83
:1013100064147004E55C6402600302127722C0E08A
:10132000C083C082C085C084C086758600C0D07569
:10133000D000C000C001C002C003C006C00790E6D4
:1013400078E030E206751B0602140890E678E0208B
:10135000E10CE51B64026006751B07021408E51B1F
:1013600024FE605F14603624FE70030213F924FC2F
:10137000700302140524086003021408AB17AA18AE
:10138000A919AF1A051A8F8275830012150E90E6FF
:1013900079F0E51A65167070751B05806B90E6791B
:1013A000E0AB17AA18A919AE1A8E82758300121520
:1013B0003B751B02E5166401704E90E678E0442010
:1013C000F08045E51624FEB51A0790E678E0442043
:1013D000F0E51614B51A0A90E678E04440F0751B63
:1013E0000090E679E0AB17AA18A919AE1A8E82759B
:1013F000830012153B051A800F90E678E04440F018
:10140000751B008003751B005391DFD007D006D0F9
:1014100003D002D001D000D0D0D086D084D085D0E7
:1014200082D083D0E032752AFF12196B90E61074D7
:10143000A0F090E611F000000090E61474E0F000D7
:101440000000E490E618F000000090E619F00000BB
:101450000090E61A7408F0000000E490E61BF0002B
:10146000000090E680E030E70F90E6247402F00080
:101470000000E490E625800DE490E624F0000000F2
:1014800090E6257440F000000043AF0190E60B7435
:1014900003F0000000D20590E68D7480F00000009B
:1014A00090E65EE04440F090E65CE0443DF07580FC
:1014B00079E4F5A0F5B075B2FF75B5F7F5B075B084
:1014C00040F5B000000090E6C07420F0000000126B
:1014D0001C2B121C4B753A01753D0175310075329C
:1014E000027536007537FC7534007535FDD2ACD207
:1014F00004C201C203752701E490E671F0F5A075FE
:10150000B4FF90E672F0F5B175B6FF021DF2BB01B3
:101510000CE58229F582E5833AF583E0225006E95D
:101520002582F8E622BBFE06E92582F8E222E58262
:1015300029F582E5833AF583E49322F8BB010DE5B2
:101540008229F582E5833AF583E8F0225006E92501
:1015500082C8F622BBFE05E92582C8F222EB9FF580
:10156000F0EA9E42F0E99D42F0EC6480C864809805
:1015700045F022EB9FF5F0EA9E42F0E99D42F0E84B
:101580009C45F022E86010ECA2E713FCED13FDEEA1
:1015900013FEEF13FFD8F022E8600FEFC333FFEE26
:1015A00033FEED33FDEC33FCD8F122D083D082F84A
:1015B000E4937012740193700DA3A393F8740193D4
:1015C000F5828883E4737402936860EFA3A3A38019
:1015D000DF300A0990E680E0440AF0800790E68058
:1015E000E04408F07FDC7E051216BA90E65D74FFD9
:1015F000F090E65FF05391EF90E680E054F7F02230
:1016000012010002000000406C15010100000102FF
:1016100000010A06000200000040010009023C002F
:1016200001010080FA0904000006FF000000070520
:101630000102400000070581024000000705020288
:1016400000020007050402000200070586020002EE
:10165000000705880200020009023C000101008029
:10166000FA0904000006FF0000000705010240001F
:101670000007058102400000070502024000000744
:1016800005040240000007058602400000070588A7
:1016900002400000040309040C034D0065006100D2
:1016A0006400650014034D0065006100640065007E
:1016B000200044005300490000008E538F5490E6F0
:1016C00000E05418700DE553C313F553E55413F5BA
:1016D00054801590E600E05418FFBF100BE5542528
:1016E000E0F554E55333F553E5541554AE53700209
:1016F00015534E6005121BB480EE22121DD0D3226A
:10170000021CD900021D1F00021D0900021CF1006D
:101710000219D500021A0C0002004200021E3C0011
:10172000021E3D00021E3E00021E3F00021E40003F
:10173000021E4100021E4200021D3500021E43002F
:10174000021E4400021E3C00021E4500021E46000E
:10175000021E4700021E4800021E4900021E4A00E7
:10176000021E4B00021E3C00021E3C00021E3C00FA
:10177000021E4C00021E4D00021E4E00021E4F00B3
:10178000021E5000021E5100021E5200021E530093
:10179000021E5400021E5500021E5600021E570073
:1017A000021E5800021E5900021E5A00021E5B0053
:1017B000021E5C00021E5D00C0E0C0F0C083C0825B
:1017C000C0D075D000C000C001C002C003C004C0BA
:1017D00005C006C007E5632401F563E43562F562E0
:1017E000E43561F561E43560F560AF67AE66AD651F
:1017F000AC64EC4D4E4F603BEF24FFF567EE34FFD9
:10180000F566ED34FFF565EC34FFF564AF67AE6661
:10181000AD65FC4D4E4F701BD209300116E53BB44F
:101820000411300005121BE98009E53864016003EA
:10183000120CCEC2CFD007D006D005D004D003D032
:1018400002D001D000D0D0D082D083D0F0D0E0320E
:1018500060801F000111133901010107010103011B
:1018600000000000F8FCFCFCFCFCFCFC000909008A
:101870000000123F011113390101010701010301A9
:1018800000000000FAFEFEFEFEFEFEFC000909005C
:10189000002D363F01113F01010101070101010047
:1018A00000000000F9FDFDFDFDFDFDFC0000001243
:1018B000002D123F01113F0101010107010111003B
:1018C00000000000FBFFFFFFFFFFFFFC0000001215
:1018D000002D363F471F80800000FC06F011007885
:1018E0007FE4F6D8FD75816B021926020FDFE493C1
:1018F000A3F8E493A34003F68001F208DFF4802903
:10190000E493A3F85407240CC8C333C4540F4420F1
:10191000C8834004F456800146F6DFE4800B0102E0
:10192000040810204080901850E47E019360BCA30E
:10193000FF543F30E509541FFEE493A360010ECF2E
:1019400054C025E060A840B8E493A3FAE493A3F858
:10195000E493A3C8C582C8CAC583CAF0A3C8C58218
:10196000C8CAC583CADFE9DEE780BE90E60174EA33
:10197000F090E6F574FFF0901F80E090E6F3F090B1
:101980001F81E090E6C3F0901F82E090E6C1F090E6
:101990001F83E090E6C2F0901F85E090E6C0F090D3
:1019A0001F86E090E6F4F075AF07741FF59A740097
:1019B000F59B759DE4E4F59EFF90E67BE090E67C68
:1019C000F00FBF80F4000000E490E6C4F0000000D7
:1019D00090E6C5F022C0E0C083C08290E680E0308F
:1019E000E70E85080C85090D85100E85110F800CFA
:1019F00085100C85110D85080E85090F5391EF9008
:101A0000E65D7410F0D082D083D0E032C0E0C083B5
:101A1000C08290E680E030E70E85080C85090D85D0
:101A2000100E85110F800C85100C85110D85080E88
:101A300085090F5391EF90E65D7420F0D082D0833A
:101A4000D0E032E490E6CEF000000090E6CFF00067
:101A5000000090E6D0F0300419121AE47FE87E030B
:101A60007D007C00121D923009FD120D1BC2041274
:101A70001C0AC202753B01D2012290E678E020E602
:101A8000F9C2E990E678E04480F0EF25E090E6794D
:101A9000F090E678E030E0F990E678E04440F090AD
:101AA000E678E020E6F990E678E030E1D6D2E92267
:101AB000A90790E678E020E6F9E51B702590E67826
:101AC000E04480F0E925E0440190E679F08D16AF1E
:101AD00003A9077517018A188919E4F51A751B03FC
:101AE000D322C322E4F55AF55BC20A200A277F04F9
:101AF0007E007D007C00121D92AF5BAE5A120D2756
:101B0000300905120D21D20A3009FD055BE55B7035
:101B1000DA055A80D622A90790E678E020E6F9E5B2
:101B20001B702390E678E04480F0E925E090E679A8
:101B3000F08D16AF03A9077517018A188919E4F506
:101B40001A751B01D322C32290E682E030E004E044
:101B500020E60B90E682E030E119E030E71590E6F0
:101B600080E04401F07F147E001216BA90E680E017
:101B700054FEF022A907AE14AF158F828E83A3E026
:101B800064037017AD0119ED7001228F828E83E01E
:101B90007C002FFDEC3EFEAF0580DF7E007F002243
:101BA00090E682E044C0F090E681F04387010000B7
:101BB000000000227400F58690FDA57C05A3E58257
:101BC000458370F922120036C201120D1BD20400A7
:101BD000000090E6047480F00000007406F000003D
:101BE00000E4F0000000D20222E535453460030233
:101BF0000C0ED3E53794FEE53694014006120C4CEA
:101C0000020BB9120C8A120BE622E4F55AF55BC3FB
:101C1000E55B9537E55A95365010121CBE121E5ED4
:101C2000055BE55B70E9055A80E522E4F563F56242
:101C3000F561F560F567F566F565F564D209F5C8F7
:101C400075CA6F75CBFED2ADD2CA227DD87C00E4B6
:101C5000FF120D7C7DC07C007F01120D7CE4FFFE35
:101C6000121DD0E4FFFE021DD9EFD39402400122E1
:101C70008F3DE53D600B146008147008120D1E8046
:101C800003120D1BD322121AB0E51B24FA600E14A6
:101C90006006240770F3D322E4F51BD322E4F51B7E
:101CA000D322121B16E51B24FA600E1460062407CB
:101CB00070F3D322E4F51BD322E4F51BD322E535E0
:101CC00045346003020B8CD3E53794FEE53694016E
:101CD0004003020BB9120BE622C0E0C083C082D2DF
:101CE000065391EF90E65D7401F0D082D083D0E08E
:101CF00032C0E0C083C082D2085391EF90E65D7499
:101D000008F0D082D083D0E032C0E0C083C08253DC
:101D100091EF90E65D7404F0D082D083D0E032C0C1
:101D2000E0C083C0825391EF90E65D7402F0D082F0
:101D3000D083D0E032C0E0C083C0825391EF90E600
:101D40005F7440F0D082D083D0E03290E7C074035B
:101D5000F090E7C27406F090E68F7403F02290E7EB
:101D600040E539F0E490E68AF090E68B04F0D32267
:101D700090E740E526F0E490E68AF090E68B04F0E8
:101D8000D322EFD394035009EF5403442090E6C0CC
:101D9000F022C2098F678E668D658C6422EFD39422
:101DA000014001228F3CD322EFD394014001228FC6
:101DB00038D322000102020303040405058F418E7B
:101DC000408D3F8C3ED322AF41AE40AD3FAC3E2272
:101DD000AD07AC067F02020D7CAD07AC067F0502A5
:101DE0000D7C90E6BAE0F539D32290E6BAE0F5260C
:101DF000D322E4F51BD2E9D2AF227F02120D3A22A0
:101E00007F05120D3A22121DD9D32253D8EF321278
:101E10001DFA22121E00228F3AD3228F33D322AF13
:101E20003D22AF2822AF3C22AF3322AF3822D3224B
:101E3000D322D322D322D322D322D322323232321C
:101E40003232323232323232323232323232323272
:101E50003232323232323232323232323232223173
:101E6000FD087F429F20A8F107A8AAA468003B00B4
:101E70007305DD207043DF64FF083B853B867615E4
:101E8000D7005B1A4D2D0D28EB40F3803A6687533F
:101E9000AA40160CFD0B350C3E41EF39D37CC40A29
:101EA000CF40250BFB54D7227C18DBD77E20FF2F99
:101EB000D7509F40EEE17D80FC05D5A0BB407ECB96
:101EC000EE606B80D708D328FF41DD0473013541F4
:101ED000BB00FA07ED04FFC8D73559A3FC021D4823
:101EE000654AFF003D80EA8A7F399700B7026FF0AC
:101EF0005DB1B332E2A57D13BA21B4D86F53ED8042
:101F00000111133901010107010103010000000063
:101F1000F8FCFCFCFCFCFCFC000909000000123F82
:101F20000111133901010107010103010000000043
:101F3000FAFEFEFEFEFEFEFC00090900002D363F03
:101F400001113F0101010107010101000000000032
:101F5000F9FDFDFDFDFDFDFC00000012002D123F0E
:101F600001113F0101010107010111000000000002
:101F7000FBFFFFFFFFFFFFFC00000012002D363FBC
:101F8000800000FC06F011221F8FD66053C1B4E41C
:101F90005680FE088B606D2897EFDF0428FDFDB6A4
:101FA00089006C407B75CF7CFD0C7AA0FB44D5C6C4
:101FB000C70876018F32BF05DB0CDF19F910F80274
:101FC0007719CF352D5AC7007F84B993AC307F0A7B
:101FD000DB57338CFE60AE68F210EF68F1ADEE5B5C
:101FE000DC1FF87C9F219E582818A634ED103FF185
:101FF000F76CED12DB41CF07FA24BF00FB092F90ED
:00000001FF
